:1000000012C01FC01EC05DC01CC01BC01AC019C0DA
:1000100018C017C016C015C079C013C012C011C0D7
:1000200010C00FC00EC011241FBECFEDCDBF10E019
:10003000A0E6B0E001C01D92AF3CB107E1F702D0ED
:1000400060C1DECF07D0789401C028D021D08823AA
:10005000E9F3FBCF82B38C6082BB80B38470809362
:10006000CC0080B388708093CD008FE189B9539A1A
:1000700083B1866083B984E088B98FEF91E09BBD3E
:100080008ABD89E08EBDBA9A88E088BF89BF08958D
:100090008091C6009091C70089270895E091C7001C
:1000A0009E2F9F5F943618F090E001C000005D9B8A
:1000B000FDCFF0E0E05AFF4F80818CB99093C700EC
:1000C00008951F920F920FB60F9211242F933F9312
:1000D0008F939F9324B535B5C9018050914097FF08
:1000E00003C0C90180509F4F99BD88BD8AE08093AD
:1000F000C90080E288BF459B89BF9F918F913F9146
:100100002F910F900FBE0F901F9018951F920F9276
:100110000FB60F9211242F933F934F935F936F93DA
:100120008F939F93EF93FF9368B160728091C900A2
:1001300081508093C900882371F0893021F46623AF
:1001400009F0CFC0D0C08091C80086956111806849
:100150008093C800C8C03091C4008091CC00E32FC8
:10016000EF5F8823C9F15E2FE43608F050E040913C
:10017000C800242F22952F70822F90E00A971CF43C
:10018000822F805D02C0822F895CE32FF0E0E05A6D
:10019000FF4F8083352F3F5F343609F430E0842FE2
:1001A00090E08F709070242F2F700A971CF4822F8C
:1001B000805D02C0822F895CE52FF0E0E05AFF4F9E
:1001C0008083232F2F5F243609F420E0E32FF0E013
:1001D000E05AFF4F80E20AC02E2FE43608F020E0FC
:1001E000E32FF0E0E05AFF4F8091C8008083209316
:1001F000C4003091CA003F5F3093CA00662309F003
:100200006EC08091CE0081508093CE008F5F39F414
:1002100083E08093CE0088B394E0892788BB8091E7
:10022000CD00811183E08093CB00381770F480916A
:10023000CC00882319F08091C6004DC08091C50084
:100240008F5F843608F447C045C08091CC00922F60
:100250009F5F8823D9F0292F943609F420E0E0919C
:10026000C400F0E0E05AFF4F8DE08083922F9F5F43
:10027000943609F490E0E22FF0E0E05AFF4F8AE074
:1002800080839093C4009093C60027C0E091C5007E
:10029000F0E0E05AFF4F3083E091C400E093C600E5
:1002A000292F943609F420E0F0E0E05AFF4F8AEA63
:1002B0008083922F9F5F943609F490E0E22FF0E064
:1002C000E05AFF4F85E580839093C500892F8F5FAB
:1002D000843609F480E08093C4001092CA0088E05C
:1002E00088BF88E089BFFF91EF919F918F916F91B7
:1002F0005F914F913F912F910F900FBE0F901F90E4
:060300001895F894FFCFF0
:00000001FF
